S018000064656D6F70726F675F786D63313430302E7372656343
S315100030000040002081400010000000000000000079
S315100030100018040000010000EE11AA5500B5E221C7
S3151000302049004058C02189000140002901D10120E2
S3151000303000E00020C0B200BD30B4C9B2D2B2140450
S315100030400C43DBB21D062543E2246400055130BC57
S315100030507047016840220A430260704701684022A7
S3151000306091430160704700B5814200D3080000BD4E
S3151000307000B5884200D3080000BDF1B588B00E0037
S315100030800C250C24002007900120059000200690A6
S31510003090002004909B48009001200500412D4BD242
S315100030A030680A214843290000F006FA0390039875
S315100030B0716800F001FA070038000A2100F007FADB
S315100030C0062906D338000A2100F0F6F907007F1CFE
S315100030D004E038000A2100F0EFF90700002F06D0AF
S315100030E003980A21794300F0E7F9029006E0039865
S315100030F00A2100F0E1F90290012007000298716898
S31510003100884204D302987168401A019003E07068EF
S315100031100299401A0190152F0CD2019800998842F5
S3151000312008D207950497019800900198FA21890012
S31510003130884201D36D1CB1E772480090402004000C
S31510003140032C1AD32000401C6E494843049900F002
S31510003150B3F93289904203D33289821A110002E000
S315100031603289121A1100009A914201D205940091E7
S315100031703289904201D3641EE2E704980599401AF9
S31510003180401E06900898FFF764FF0698401E01033C
S31510003190E020C00108407189491E8A01C0211140F2
S315100031A001430598401E0002F022120102400A4314
S315100031B00798401E8006800E1043089908610898EB
S315100031C0FFF74CFF09B0F0BD70B505000C001600F6
S315100031D02800FFF723FF0028FAD023005B1CDBB280
S315100031E03200D2B202212800FFF726FF70BD10B5BB
S315100031F004008020800300F098F92068012188439C
S31510003200206020688007FCD410BD38B5040020006B
S3151000321000F085F8012802D0022804D007E000F05B
S3151000322097F9050005E000F09DF9050001E0002082
S315100032300500280032BDF6B589B006003000FFF74C
S31510003240D6FF09A80178300000F05EF83000FFF7CD
S31510003250DCFF01908021C900009101980A9900F0C5
S315100032602BF90099091A0020FFF7FDFE6F49FFF7A9
S31510003270FFFE059001988021C900059A891A00F071
S315100032801BF907900A988009069001988009029008
S315100032906649009106988021C9004843029900F0BA
S315100032A00BF90099FFF7E4FE04900298049948433D
S315100032B0800A0700BF010A98C01B0A99079A891A43
S315100032C0884201D3012400E00024E4B2002C02D08D
S315100032D00598039001E004980390E4B2002C01D005
S315100032E0012500E00225F06851490140F160F068BF
S315100032F0EDB2A903039A0A430243F2600BB0F0BD84
S315100033000000000010270000E422520082580F230C
S315100033109A43C9B20A43E4235B00C2507047E421C2
S31510003320490040580007000F7047F8B504002068A0
S315100033305C4940184709780940033902F826760196
S315100033400E40064320688068574901402068816016
S31510003350206880683043216888606068800002D5E4
S31510003360606880003BD5207E002802D0207E012890
S3151000337035D120202168C861606801008900C90F15
S31510003380002914D1606805006D0F6D07290060686B
S3151000339085040D4320688561A06805006D0F6D07D3
S315100033A02900A06885040D432068C56005E06068A3
S315100033B021688861A0682168C860207E012807D12D
S315100033C0200000F00DF8802000052168C86103E098
S315100033D0802000012168C86134482168C861F1BDA8
S315100033E010B5010003200A7E012A1AD120220B688B
S315100033F0DA610A6812682E4B13400A7B1206F02413
S31510003400240514401C430A6814600A690B681A6183
S315100034104A690B685A61274A0B68DA610022100064
S3151000342001E003221000C0B210BD0000FF0300002F
S31510003430003CFFFFF0B501000120002200230C68BC
S31510003440E5692C002405E40F0D68EE6935006D075B
S31510003450ED0F002C02D00326300020E0012D02D102
S31510003460022630001BE00E6836690E610E6876691A
S315100034704E610E68F669B6083700FF07FF0F3A006F
S315100034800E68F669F6083700FF07FF0F3B00D2B249
S31510003490002A02D0DBB2002BE5D100263000C0B2E4
S315100034A0F0BD000000F0FBAFFF00FFFF4000A006DC
S315100034B0FFFFFFF040002800020004200F4B1860A9
S315100034C00F4802600F48016010480068704770B5D9
S315100034D002000B00042009490860094802600948E7
S315100034E003600948006800210100002004000D0057
S315100034F00648006800212043294370BD340003406C
S3151000350020000340240003402C0003402800034001
S31510003510C3200E490860704700B5C0200B490860EB
S315100035200A4800684007FBD400BD10B50400FFF739
S31510003530F3FF0A48006820430849086006480068F7
S315100035404000FBD4FFF7E4FF10BD0000240001404B
S315100035500348006870470000000301401003014053
S31510003560D401002000487047002D310100B5BFF38B
S315100035704F8F8248CB490860BFF34F8F00BFFDE7DE
S3151000358010B4C9B204234B43C318DB690724A34301
S31510003590D2B21343C9B204244C430419E36110BCDC
S315100035A070478A2149004058C1080800C007C00F5B
S315100035B07047016C0F22914302220A43026470473E
S315100035C070B504000D001600EDB2042068432018F3
S315100035D0C06950218843EDB2042169436118C8615E
S315100035E03200D2B22900C9B22000FFF7C9FF70BD60
S315100035F0C26807239A43C9B24B075B0F1343C360D4
S315100036007047016840220A430260704701684022F1
S31510003610914301607047016801220A4302607047B6
S31510003620016801229143016070470068C0697047C4
S315100036300268D161704780B500F00DF800F0A0F86F
S3151000364001BD80B500F045F800F02EF901BD80B53A
S31510003650FFF78CFF01BD00B587B0E1200002009096
S315100036600820694608710820694648710120694694
S31510003670887110206946C87100206946088169461C
S31510003680A34800F065F900206946087505AA0321CC
S31510003690A04800F0F1F99C206946087303AA02219C
S315100036A09C4800F0E9F9002200219948FFF788FFAD
S315100036B0012304221021964800F0B7FA01230422B0
S315100036C00021934800F0CAFA9148FFF772FF07B03D
S315100036D000BD80B590480078002813D18F4800F0BF
S315100036E03EF801283AD18D480078002836D000F0EF
S315100036F062FB8B49086001208749087000208949C0
S3151000370008702BE08548874909784018401C00F05E
S3151000371026F8012818D183480078401C8149087082
S31510003720804800787D490978884217D100207A4967
S3151000373008707A484078FF2810D178488078002899
S315100037400CD1FFF784FF09E000F035FB74490968D6
S315100037506431814202D200206F49087001BD10B554
S3151000376004006B48FFF71DFF002805D1684800F0DC
S3151000377031F92070012000E0002010BD0400FA0588
S3151000378030B587B0FFF7E4FE04006748844202D2E2
S3151000379002204443F9E76548844201D36408FAE7F6
S315100037A0220001216248FFF746FD0094614801900E
S315100037B0FA20400169460881012069464881694618
S315100037C05D48FFF75AFC5C48FFF71BFF5A48FFF7A6
S315100037D022FF5A485A4908605948406880008008B4
S315100037E08021090601435648416055484068400FFC
S315100037F04007544901435248416051488068400F80
S315100038004007504901434E4881604D4840684E4933
S3151000381001404B4841604A48806880218905014330
S315100038204748816008204649087300200500280093
S315100038304349097BC0B2884206D200204049EDB206
S31510003840491908746D1CF2E700203D4908763C487A
S31510003850FFF76BFD012201213548FFF7B5FC36480D
S31510003860FFF7D4FE3448FFF7DBFE002069460875E3
S3151000387005AA0821354800F0FFF8A4206946087308
S3151000388003AA0921314800F0F7F82B48FFF7B9FED3
S3151000389002212948FFF7ACFE2748FFF7B7FE07B00D
S315100038A030BD00000CED00E030B583B00025244893
S315100038B0FFF7BBFEC0071BD52148FFF7BBFD00284D
S315100038C012D10020040020001D49097BC0B2884295
S315100038D00AD21B48E4B20019007C6946E4B20855C6
S315100038E001200500641CEEE701211548FFF7A0FE34
S315100038F0EDB2012D0BD10020050068460078FF2897
S3151000390005D168464078002801D1FFF7A0FE37BDE3
S315100039100002004800010440D1010020540100209B
S3151000392098010020D0010020001BB700010E2707C8
S315100039300000045020A1070000030450201004507A
S31510003940A001002067060000FFFFFFDF000404400F
S3151000395070B504000E001025200000F0EFF8F07985
S31510003960002801D0F07905002A003168200000F007
S3151000397005F9B079401E40002900891CC901FF22B3
S315100039809143014312480843E0633079401E000614
S3151000399081214900014361637079002806D0606B6C
S315100039A07179491E09040143616305E0606B317941
S315100039B0491E090401436163A020C000A0630020D2
S315100039C0C043E0640820305E206470BD0000000033
S315100039D00100030000B50100862252008A58E02338
S315100039E0DB041340002B02D14A6D100003E08E2237
S315100039F052008A58100080B200BDF8B4016842180F
S31510003A0043685908511800918168DB0701D54B4668
S31510003A10C918009B9A4202D10C30F2BC7047137839
S31510003A20521C032403261E4002D11678F61C521C83
S31510003A301D090F2D07D115780F35521C03E0177885
S31510003A40521C0F70491C761EF9D1002DE1D0167844
S31510003A50521C9B081C40032C01D11478521C2302C3
S31510003A60F3185C420B19AD1CD3D01C785B1C0C7080
S31510003A70491C6D1ECDD0F8E7F0B5C9B28B100424E1
S31510003A806343C318C9B28C1004256C430419246906
S31510003A90FC258E07B60F08277E43B540AC431C6144
S31510003AA0436F03244D00AC40A3434367C9B2CB0810
S31510003AB004246343C318C9B2CC0804256C43041903
S31510003AC0246C04254E07760F04277E43B540AC437D
S31510003AD01C64C9B2CB0804246343C318C9B2CC080A
S31510003AE004256C430419246C55784F077F0F042660
S31510003AF07743BD4025431D640F4B984204D1036E96
S31510003B0001248C40A343036653688B404360C9B2BB
S31510003B108B1004246343C318C9B28C1004256C435C
S31510003B200419246915788F07BF0F08267743BD40FF
S31510003B3025431D61F0BD00000002044010B50400CD
S31510003B409020C005844202D05B48844203D15B4872
S31510003B5000F0A0F808E05A48844202D0594884423E
S31510003B6002D1594800F096F80320E060E068C007DB
S31510003B70FCD5206C0F218843206410BDF0B589B0A8
S31510003B8007000D001600642D48D3002E46D0FFF70F
S31510003B90DFFC6421FFF790FC079028006421FFF7F3
S31510003BA08BFC0500012005900120029047480090EB
S31510003BB046480400002C1DD0079860432900714325
S31510003BC0FFF77AFC04900498800A03900498800505
S31510003BD0800D019003988021C900884208D201986F
S31510003BE00099884204D20198009003980290059497
S31510003BF0641EDFE70598802109020143396178695F
S31510003C0033490140701E800208430299491E090477
S31510003C100143796100206946087602E00120694671
S31510003C2008766846007E09B0F0BD30B4842464007E
S31510003C300459284D254084246400055184246400C9
S31510003C400459254D25401C022C430C43D2B21506AF
S31510003C50254384246400055130BC704730B4862453
S31510003C60640004591B4D25408624640005518624A2
S31510003C7064000459194D25401C022C430C43D2B242
S31510003C8015062543802464052C4386256D00445172
S31510003C9030BC704710B504000848844203D1082090
S31510003CA0FFF743FC06E00848844203D18020C00297
S31510003CB0FFF73BFC10BD000000020048080000485A
S31510003CC0004000480042004808400048FF0300003A
S31510003CD0EF8000FCFFFFFFF8C0C0FFF8C0C0FFEF89
S31510003CE0F0B540B2002821D5374C40B20207120F6A
S31510003CF0083A950804225543334A40B203071B0F6E
S31510003D00083B9B0804267343D258FF238607B60F39
S31510003D1008277E43B3409A438B01DBB28607B60F62
S31510003D2008277E43B340134363511AE0274A40B233
S31510003D30830804246343D258FF238407A40F08255D
S31510003D406C43A3409A438B01DBB28407A40F08256A
S31510003D506C43A34013431D4A40B2840804256C43A8
S31510003D601351F0BD10B50400601E8021490488422D
S31510003D7001D301200EE0601E1549086003210020C2
S31510003D80C043FFF7ADFF0020124908600720124913
S31510003D900860002010BD80B510480068FA2189001F
S31510003DA0FFF78AFBFFF7DEFF002000F001F801BDE8
S31510003DB00B49086070470A48006870470848006851
S31510003DC0401C0749086070471CED00E000E400E065
S31510003DD014E000E018E000E010E000E0D40100205C
S31510003DE0CC01002080B523480068000AC0B22249E1
S31510003DF008602148006800282FD01E480068C0B20D
S31510003E001E4908601D4800681D4909680902C0223C
S31510003E1092000A400243194802601948006880055A
S31510003E200CD41848144909688902144A126889186A
S31510003E30FFF742FB0001144908601AE0FFF792FBF6
S31510003E4080010D49096889020C4A12688918FFF722
S31510003E5033FB00010C4908600BE009480068800537
S31510003E6003D40A480849086003E0FFF77BFB0649BC
S31510003E70086001BD00030140C4010020C8010020F4
S31510003E801C03014000001BB7D4010020006CDC02AB
S31510003E9013008B404360704780B58022002116487E
S31510003EA000F030F8012200211348FFF7F1FF01BDA1
S31510003EB010B5FFF780FF040010480068201AFA2199
S31510003EC04900884217D30E480078002809D10120EE
S31510003ED00B4908708022520200210748FFF7D8FFCD
S31510003EE007E0002006490870012200210248FFF76A
S31510003EF0CFFF0248046010BD00040440C00100203A
S31510003F00D2010020F0B4C9B28B0804246343C3184D
S31510003F10C9B28C0804256C4304192469FC258E0744
S31510003F20B60F08277E43B540AC431C61C9B28B0857
S31510003F3004246343C418C9B28B0804256B43C31801
S31510003F401D69D2B28E07B60F08235E431300B34025
S31510003F502B432361F0BC704780B5C0200849086028
S31510003F6008480068084901400648016007480849A2
S31510003F700860C32002490860FFF734FF01BD00BF87
S31510003F80240001401C030140FFFDFFFF0001F13F2B
S31510003F900003014070B40121002213E00468001DE3
S31510003FA00C4202D04D466D1E64192260241D1B1F43
S31510003FB0042BFAD225009E0701D52280AD1C0B409A
S31510003FC000D02A700368001D002BE7D170BC704723
S31510003FD010B5074979441831064C7C44163404E070
S31510003FE0081D0A68891888470100A142F8D110BD3A
S31510003FF008000000240000009DFFFFFF8000000065
S315100040005401002000000000F3F9FFFFFC0000003F
S315100040102E0100000C00002080B500F007F8FFF715
S315100040200AFBFFF745FFFFF70CFBFAE780B5FFF732
S3151000403033FFFFF7B0FE01BD00F00BF8002801D0EA
S31510004040FFF7C6FF002000BF00BFFFF7E5FF00F037
S3151000405002F80120704780B500F002F801BDFEE7B6
S315100040600746384600F002F8FBE7FEE780B500BFCA
S3151000407000BF024A11001820ABBEFBE72600020063
S315100040800248854602488047024800470040002003
S31510004090AD400010B9400010034800680121884364
S315100040A001490860704700BF6800014080B5FFF7FE
S315100040B0F3FFFFF751FF01BD00BF00BF00BF00BFF8
S315100040C0FFF7BAFFFEE7FEE7FEE7FEE7FEE7FEE7CD
S315100040D0FEE7FEE7FEE7FEE7FEE7FEE7FEE7FEE7A2
S315100040E0FEE7FEE7FEE7FEE7FEE7FEE7FEE7FEE792
S315100040F0FEE7FEE7FEE7FEE7FEE7FEE7FEE7FEE782
S31510004100FEE7FEE7FEE7FEE720022C480047041212
S315100041102B04122A041229041228041227045226E8
S3151000412004122404522308F1730410036B40001088
S315100041305F0412C50412C7041003BD3D0010C90860
S3151000414012CB0412CD0412CF0412D10412D30412CE
S31510004150D50412D70412D90412DB0412DD0412DFBF
S315100041600412E10412E30412E50412E70412E9044E
S3151000417012EB0412ED0412EF0412F10412F30412FE
S31510004180F50412F70412F90412FB0412FD0412FFCF
S3141000419004100301410010030412050412070462
S705100040B9F1
